:100000002EC03BC03AC039C038C037C036C035C03A
:1000100034C033C032C031C030C02FC02EC08AA21D
:10002000B0BAC3FFA3A3A3A1A1A1A1A1A1A3A3A30C
:10003000A3A3A1A1A1A1A114E6FF00000000000359
:10004000146EFFFFFF000000000000005AFFFCFEDE
:10005000FDFF000000073889FFFCFEFDFF001124B2
:100060001FBECFEDCDBF10E0A0E6B0E001C01D92F5
:10007000AC36B107E1F7D0D0BBC1C2CF20ED37E03D
:1000800003C0F9013197F1F70197D8F7089588EE89
:1000900093E0F4CFCF93C09163008C2F8F5F8F7765
:1000A00080936300909161009295990F907E60918A
:1000B00062006295660F660F607C692B909160000C
:1000C000692B90E087D16FEF8C2F90E0CF9182C1A8
:1000D000CF931092630008C08C2F90E073D18F3FB4
:1000E00041F4CF5FC0936300C0916300C7FFF4CFBA
:1000F0000EC0982F9F709093600085FB992790F910
:100100009093610086FB882780F980936200CF91ED
:10011000089580916100811112C087E0809366008C
:1001200082E590E090936A00809369008FE390E00D
:1001300090936800809367008CE290E011C084E0A7
:10014000809366008AE490E090936A00809369004F
:1001500087E390E0909368008093670084E290E0EA
:100160009093650080936400809166008C5F80931B
:100170006B000895811104C0611102C091EA9ABD1B
:1001800088BD69BD089590E0E0916400F09165003C
:10019000E80FF91FE491EABDE0916700F091680073
:1001A000E80FF91F6491E0916900F0916A00E80F8F
:1001B000F91F8491DFCF369A3699FECF85B1089525
:1001C0001F93CF93DF93C82F14E1D1EA0CC018BC62
:1001D00019BD84E690E052DFDABD18BC19BC80E995
:1001E00091E04CDFC150C111F2CFDF91CF911F914F
:1001F00008951F93CF93DF93EC01888111E081274D
:10020000888348DF82E0DCDF88818127888342DFC2
:10021000DF91CF911F913BCFA39A83EA87B986ECF8
:1002200086B93699FECF369A3699FECFC5B1B99ABE
:10023000B89A81EA8ABD81E083BF4ADF6ADFCF3B9B
:1002400080F080916C008F5F8F7180936C00809143
:1002500060008F5F80936000909166008917D0F0F6
:1002600017C010926C00CF3578F0809160009091AB
:100270006600891301C00CC0811102C080916B001F
:1002800081508093600006C080916200811102C09D
:1002900010926000FFDEBB9AC39AA29A81EA87B9E6
:1002A00086EC86B9369AC0E010E00FEF81EAF82EAE
:1002B00080916000E0916900F0916A00E80FF11D03
:1002C000D49190916C00903160F0E1DE10926C005E
:1002D0001092600081E690E08CDF82E690E089DF9A
:1002E00044C0DD3F59F408BD19BC82E390E0C6DE8E
:1002F000FABC18BC19BC82E390E011C0DC3F89F461
:10030000D4E008BD19BC85E090E0B8DE18BC09BD9A
:1003100081E490E0B3DED150A1F780ED92E0AEDE53
:1003200024C0DE3F81F447DF982F80E001C08F5F5B
:10033000E82FF0E0E25EFF4FE491E917C0F340DF01
:10034000A6DEA5DE12C01FDF1F5F1B3548F0DF3FB2
:1003500039F48091660082508093600014DF9ADE49
:1003600084EF91E08BDE10926C00349BA1CF85B1BD
:10037000813828F5CF5FC83018F1C09160008091B6
:100380006600C81798F4CC2311F0C15010C0FABC15
:1003900018BC19BC85B7877E806185BF85B7806230
:1003A00085BF889585B78F7D85BF01C0C2E08C2F42
:1003B000EADEC09360006EDE8AEF90E05FDEC0E0B0
:1003C000369A76CFE199FECF1FBA8EBBE09A992775
:1003D0008DB30895262FE199FECF1CBA1FBA8EBBAC
:1003E0002DBB0FB6F894E29AE19A0FBE01960895DC
:0403F000F894FFCFAF
:00000001FF
